:02000000CB290A
:080008000900813086000F3071
:1000100085000F308500C0308600080082308600E1
:100020000F3085000F308500C03086000800843016
:1000300086000F3085000F308500C0308600080034
:10004000883086000F3085000F308500C030860074
:100050000800903086000F3085000F308500C030DA
:1000600086000800A03086000F3085000F30850024
:10007000C03086000800413086000F3085000F3008
:100080008500C03086000800423086000F308500B1
:100090000F308500C03086000800443086000F30E5
:1000A00085000F308500C03086000800483086008B
:1000B0000F3085000F308500C030860008005030BA
:1000C00086000F3085000F308500C03086000800A4
:1000D000603086000F3085000F308500C03086000C
:1000E0000800C13086000E3085000F308500C0301A
:1000F00086000800C23086000E3085000F30850073
:10010000C03086000800C43086000E3085000F30F5
:100110008500C03086000800C83086000E3085009B
:100120000F308500C03086000800D03086000E30C9
:1001300085000F308500C03086000800E030860062
:100140000E3085000F308500C03086000800C130B9
:1001500086000D3085000F308500C0308600080015
:10016000C23086000D3085000F308500C03086001B
:100170000800C43086000D3085000F308500C03087
:1001800086000800C83086000D3085000F308500DD
:10019000C03086000800D03086000D3085000F305A
:1001A0008500C03086000800E03086000D308500F4
:1001B0000F308500C03086000800C13086000B304B
:1001C00085000F308500C03086000800C2308600F0
:1001D0000B3085000F308500C03086000800C43029
:1001E00086000B3085000F308500C0308600080087
:1001F000C83086000B3085000F308500C030860087
:100200000800D03086000B3085000F308500C030EC
:1002100086000800E03086000B3085000F30850036
:10022000C03086000800C1308600073085000F30DE
:100230008500C03086000800C23086000730850087
:100240000F308500C03086000800C43086000730BB
:1002500085000F308500C03086000800C830860059
:10026000073085000F308500C03086000800D03090
:100270008600073085000F308500C03086000800FA
:10028000E0308600073085000F308500C0308600E2
:1002900008008207532959296429732983298D2944
:1002A0009F29AE29BD2983208D0B53298E0B5329FD
:1002B00008004D207A20B0208320C2208C208D0B96
:1002C00059298E0B59290800172044207120A72096
:1002D000E620B920F820CB20952056208D0B6429EC
:1002E0008E0B64290800F820EF20E620DD20B020E6
:1002F00083205620202017200E2005208D0B7329E7
:100300008E0B73290800EF20B92083204D20172081
:100310008D0B83298E0B83290800F820C2208C20A6
:100320005620202017200E2005203B207A208320F5
:10033000B020EF208D0B8D298E0B8D290800EF202A
:10034000E620A72071203B200E20172056208C206D
:10035000C2208D0B9F298E0B9F290800F820DD20DD
:10036000A72071203B200E20172056208C20C22071
:100370008D0BAE298E0BAE2908000121C2208320EF
:1003800044200520DD20B020562029208D0BBD29DA
:100390008E0BBD29080083160030850000308600D2
:1003A00083128C018D018E01E030860007308500BC
:1003B00050308D008E0001308A000C08EA218F0039
:1003C00001308A000F0849218C0A0C08F73E0318F7
:1003D0008C01D829820700340134023403340434F8
:0803E00005340634073408342B
:02400E00F33F7E
:00000001FF
